:020000040800F2
:1000000000500020C90A0008910A0008990A000857
:1000100000000000000000000000000000000000E0
:10002000000000000000000000000000E1320008B5
:10003000000000000000000001340008A10A0008D0
:10004000190B0008190B0008190B0008190B000800
:10005000190B0008190B0008190B0008190B0008F0
:10006000190B0008190B0008190B0008190B0008E0
:10007000190B0008190B0008190B0008190B0008D0
:10008000190B0008190B0008190B000800000000EC
:10009000190B0008190B0008190B0008190B0008B0
:1000A000190B0008190B0008190B0008190B0008A0
:1000B000190B0008190B000800000000190B0008BC
:1000C00010B5064C2378002B07D1054B002B02D02E
:1000D000044800E000BF0123237010BD1000002081
:1000E000000000006C380008044B10B5002B03D052
:1000F0000349044800E000BF10BDC04600000000F6
:10010000140000206C380008002243088B4274D38E
:1001100003098B425FD3030A8B4244D3030B8B4208
:1001200028D3030C8B420DD3FF22090212BA030C11
:100130008B4202D31212090265D0030B8B4219D3F2
:1001400000E0090AC30B8B4201D3CB03C01A524112
:10015000830B8B4201D38B03C01A5241430B8B425A
:1001600001D34B03C01A5241030B8B4201D30B0343
:10017000C01A5241C30A8B4201D3CB02C01A52416A
:10018000830A8B4201D38B02C01A5241430A8B422D
:1001900001D34B02C01A5241030A8B4201D30B0216
:1001A000C01A5241CDD2C3098B4201D3CB01C01A30
:1001B000524183098B4201D38B01C01A524143093A
:1001C0008B4201D34B01C01A524103098B4201D328
:1001D0000B01C01A5241C3088B4201D3CB00C01A95
:1001E000524183088B4201D38B00C01A524143080D
:1001F0008B4201D34B00C01A5241411A00D2014632
:10020000524110467047FFE701B5002000F006F8A4
:1002100002BDC0460029F7D076E770477047C04658
:10022000002B11D1002A0FD1002900D1002802D0C3
:100230000021C943080007B4024802A140180290F7
:1002400003BDC046D9FFFFFF03B4684601B502985D
:1002500000F034F8019B9E4602B00CBC7047C046CB
:10026000F0B5CE469946030C9C46130447461B0C3A
:100270001D000E0061460404240C80B50700100C1C
:100280004B436543414360432C0CC01824188C46F3
:10029000A34203D980235B029846C444494679436C
:1002A0005643230C2D042D0C891963442404601932
:1002B000C918C0BCB946B046F0BDC046F0B55746F7
:1002C0004E464546DE46E0B504000D00924699468E
:1002D00083B08B4230D82DD04946504600F0D8F834
:1002E00029000600200000F0D3F8331A9846203B7E
:1002F00034D49B4653465A46934042461F005346C9
:1003000093401E00AF423BD8AF4200D179E05B463C
:10031000A41BBD41002B00DA76E0002200230092EE
:10032000019301235A46934001930123424693408F
:10033000009329E08242CFD900220023009201934A
:100340000C9B002B01D01C605D600098019903B0EC
:10035000F0BCBB46B246A946A046F0BD42469B460D
:1003600020239B1A5246DA40414613004A468A40EF
:10037000170042461F43534693401E00AF42C3D965
:1003800000220023009201934346002BD8D0FB07A4
:1003900072081A4346467B080EE0AB4201D1A242E6
:1003A0000CD8A41A9D41012024196D410021013E61
:1003B00024184D41002E06D0AB42EED9013E24193F
:1003C0006D41002EF8D1009801995B4600196941F2
:1003D000002B24DB2B005A464446D3402A00E2403F
:1003E0001C005B461500002B2ADB26009E403300D4
:1003F00026004746BE403200801A99410090019184
:100400009EE7A342BCD882E74246202300219B1AE4
:100410000022009101920122DA40019285E74246D2
:1004200020239B1A2A0046469A402300F340444664
:1004300013432A00E2401C005B461500002BD4DA6F
:1004400042462F002023260097409B1ADE403B00A7
:100450003343CDE71C2101231B04984201D3000C38
:1004600010391B0A984201D3000A08391B09984227
:1004700001D30009043902A2105C40187047C0463D
:10048000040302020101010100000000000000005D
:1004900010B5002903D1FFF7DDFF203002E008008E
:1004A000FFF7D8FF10BDC04680B584B000AFF8603C
:1004B000B9607A60FB68064A1A60BB68054A1A6030
:1004C0007B6880221A60C046BD4604B080BDC0462D
:1004D0002C0000208000002080B584B000AFF860C0
:1004E000B9607A603B608023DB0563229A628023D7
:1004F000DB054022FF32DA6200220021002000F0FA
:1005000015F8094B0021180001F012FC064B0421DC
:10051000180001F00DFC044B0821180001F008FC44
:10052000C046BD4604B080BD8802002090B587B0AB
:1005300000AF040008001100FB1D221C1A70BB1D37
:10054000021C1A707B1D0A1C1A70FB1D1A781300FE
:100550009B009B189B0100D5FF331B127B61BB1DC9
:100560001A7813009B009B189B0100D5FF331B12C8
:100570003B617B1D1A7813009B009B189B0100D5E3
:10058000FF331B12FB608023DB057A695A638023EB
:10059000DB053A699A638023DB05FA68DA63C046B3
:1005A000BD4607B090BD000080B586B000AF786052
:1005B0000023002200210020FFF78EFF00237B6133
:1005C00000233B61464B00221A70A023DB058021EB
:1005D000180000F045FD03005A425341DAB20F23E0
:1005E000FB181A70A023DB054021180000F038FD2D
:1005F00003005A425341DAB20E23FB181A70A023AB
:10060000DB052021180000F02BFD03005A42534166
:10061000DAB20D217B181A707B181B78002B10D1D1
:100620007B69462B05DD7B69812B02DC2C4B00228C
:100630001A703B6901333B613B69072B01DD0023E5
:100640007B610D23FB181B78012B04D100233B6138
:100650007B6901337B617B69782B02DD204B0122B2
:100660001A700E23FB181B78012B02D11C4B02229F
:100670001A700F23FB181B78012B02D1184B032291
:100680001A7000F0B1FA0300164A934202D8144BD4
:1006900000221A70124B1B78022B11D016DC002B93
:1006A00002D0012B06D011E03C220A21FF20FFF7E7
:1006B0003DFF11E03C220A21FF20FFF737FF0BE04E
:1006C000FF2200210020FFF731FF05E05A2282219E
:1006D000FF20FFF72BFFC046052002F041F874E72A
:1006E000840200200F27000080B582B002AF0649C7
:1006F0000648074B0193012300930023802202F058
:1007000033F9C046BD4680BD84380008A9050008FD
:100710008002002090B589B000AF00F0FFF900F032
:100720001FF800F00DF900F077F83B1D0A4A13CAD4
:1007300013C313CA13C312681A603B1D00211800AB
:1007400001F0C1FF0200054B1A60FFF7CDFF01F079
:10075000B2FFC046FDE7C0469C380008C802002032
:1007600090B595B000AF18243B19180038231A0033
:10077000002103F04FF83B1D180014231A0000213C
:1007800003F048F8224B1B68224A1A40204B802174
:1007900009010A431A6021007B1802221A607B18A3
:1007A0000122DA607B1810221A617B1802229A62F9
:1007B0007B180022DA627B188022D2021A637B182F
:1007C0008022D2035A637B18180000F067FC031ED6
:1007D00001D000F0E9F83B1D0F221A603B1D0322F7
:1007E0005A603B1D00229A603B1D0022DA603B1DCF
:1007F00000221A613B1D0121180001F023F8031E9D
:1008000001D000F0D1F8C046BD4615B090BDC0463D
:1008100000700040FFE7FFFF80B58AB000AF1823EB
:10082000FB18180010231A00002102F0F3FF102318
:10083000FB18180008231A00002102F0EBFF3B0010
:10084000180010231A00002102F0E4FF3A4B802226
:10085000D2051A60384B00225A60374B00229A604A
:10086000354B364ADA60344B00221A61324B002293
:100870005A61314B180001F0D3F9031E01D000F08A
:1008800093F818217B18802252011A607A182A4B9B
:100890001100180001F0A4FB031E01D000F084F841
:1008A000254B180001F0FCF9031E01D000F07CF884
:1008B00010217B1800221A607B1800225A607A18D7
:1008C0001D4B1100180001F07FFE031E01D000F047
:1008D0006BF83B0060221A603B0000225A603B002C
:1008E00002229A603B000022DA603900124B00229B
:1008F000180001F0AFFA031E01D000F055F83900DE
:100900000D4B0422180001F0A5FA031E01D000F0DF
:100910004BF83900084B0822180001F09BFA031E1F
:1009200001D000F041F8044B180000F075F8C04603
:10093000BD460AB080BDC04688020020FFFF00000F
:1009400080B586B000AF3B1D180014231A000021AB
:1009500002F060FF0F4BDA6A0E4B01210A43DA62A4
:100960000C4BDB6A012213403B603B683B1DE022DD
:100970001A603B1D00225A603B1D00229A603A1DFE
:10098000A023DB051100180000F0ECF9C046BD46BD
:1009900006B080BD0010024080B582B000AF786024
:1009A000012001F0DDFEFBE780B500AF72B6C04666
:1009B000C046FDE780B500AF0B4B5A6B0A4B0121D7
:1009C0000A435A63084B9A6B074B802149050A4337
:1009D0009A6302235B4200220321180000F0A0F971
:1009E000C046BD4680BDC0460010024080B582B002
:1009F00000AF78607B681A688023DB059A4205D1D6
:100A0000044B9A6B034B01210A439A63C046BD46CF
:100A100002B080BD0010024090B589B000AF786090
:100A20000C243B19180014231A00002102F0F2FED6
:100A30007B681A688023DB059A4222D1134BDA6A5D
:100A4000124B01210A43DA62104BDB6A0122134088
:100A5000BB60BB6821007B1807221A607B1802224A
:100A60005A607B1800229A607B180222DA607B1899
:100A700002221A617A18A023DB051100180000F089
:100A800071F9C046BD4609B090BDC0460010024095
:100A900080B500AFC046FDE780B500AFC046FDE7BA
:100AA00080B500AF00F08EF802F068FB0300012B68
:100AB00001D002F0C9FCC046BD4680BD80B500AF84
:100AC000C046BD4680BD00000D488546FFF7F6FFD5
:100AD0000C480D490D4A002302E0D458C450043399
:100AE000C4188C42F9D30A4A0A4C002301E013606F
:100AF0000432A242FBD302F095FEFFF70BFEFEE7A5
:100B0000005000200000002010000020EC380008F9
:100B10001000002014100020FEE7000080B582B015
:100B200000AFFB1D00221A700B4B1A680A4B4021C4
:100B30000A431A60032000F011F8031E03D0FB1DC6
:100B400001221A7001E0FFF735FFFB1D1B7818002A
:100B5000BD4602B080BDC0460020024090B583B0C3
:100B600000AF7860144B1C68144B1B781900FA23F3
:100B70009800FFF7C9FA030019002000FFF7C4FA34
:100B80000300180000F0E1F8031E01D001230FE07C
:100B90007B68032B0BD8796801235B420022180085
:100BA00000F0BEF8064B7A681A60002300E00123CB
:100BB0001800BD4603B090BD0000002008000020D2
:100BC0000400002080B500AF054B1B781A00054BD0
:100BD0001B68D218034B1A60C046BD4680BDC04694
:100BE00008000020CC02002080B500AF024B1B683B
:100BF0001800BD4680BDC046CC02002090B583B031
:100C000000AF02003960FB1D1A70FB1D1B787F2BA3
:100C100028D82F4AFB1D1B785BB29B08C0339B0072
:100C20009B58FA1D1278110003220A40D200FF21BE
:100C300091400A00D2431A4011003B689B01FF22F9
:100C40001A40FB1D1B78180003230340DB009A4069
:100C50001F48FB1D1B785BB29B080A43C0339B00F7
:100C60001A5031E01B4AFB1D1B7819000F230B4063
:100C7000083B9B0806339B00D31804331B68FA1DFE
:100C80001278110003220A40D200FF2191400A008D
:100C9000D2431A4011003B689B01FF221A40FB1D02
:100CA0001B78180003230340DB009A400948FB1D12
:100CB0001B781C000F232340083B9B080A43063384
:100CC0009B00C31804331A60C046BD4603B090BDF4
:100CD00000E100E000ED00E080B582B000AF786098
:100CE0007B685A1E80235B049A4201D3012310E0E3
:100CF0000A4B7A68013A5A6001235B4203211800CB
:100D0000FFF77CFF054B00229A60044B07221A6014
:100D100000231800BD4602B080BDC04610E000E0D0
:100D200080B584B000AFB9607A600F217B18021CD7
:100D30001A70BA687B181B785BB211001800FFF7B5
:100D40005DFFC046BD4604B080BD80B582B000AF37
:100D500078607B681800FFF7BFFF03001800BD46EE
:100D600002B080BD80B586B000AF786039600023E6
:100D70007B610023FB6000233B6155E13B681B68FE
:100D800001217A6991400A001340FB60FB68002B47
:100D900000D146E13B685B6803221340012B05D07C
:100DA0003B685B6803221340022B30D17B689B6851
:100DB0003B617B695B0003229A401300DA433B6985
:100DC00013403B613B68DA687B695B009A40130023
:100DD0003A6913433B617B683A699A607B685B6858
:100DE0003B6101227B699A401300DA433B6913405F
:100DF0003B613B685B681B0901221A407B699A4092
:100E000013003A6913433B617B683A695A603B6857
:100E10005B6803221340032B17D07B68DB683B61C0
:100E20007B695B0003229A401300DA433B6913405D
:100E30003B613B689A687B695B009A4013003A69A2
:100E400013433B617B683A69DA603B685B68032265
:100E50001340022B23D17B69DA087B6808329200A9
:100E6000D3583B617B69072213409B000F229A40B5
:100E70001300DA433B6913403B613B681A697B69A5
:100E800007210B409B009A4013003A6913433B61D2
:100E90007B69DA087B68083292003969D1507B6837
:100EA0001B683B617B695B0003229A401300DA43B5
:100EB0003B6913403B613B685B6803221A407B69D6
:100EC0005B009A4013003A6913433B617B683A69BF
:100ED0001A603B685A68C0239B02134000D1A0E00F
:100EE000574B5A6B564B01210A435A63554A7B694B
:100EF0009B0802339B009B583B617B690322134094
:100F00009B000F229A401300DA433B6913403B6178
:100F10007A68A023DB059A421FD07B684A4A934235
:100F200019D07B68494A934213D07B68484A934260
:100F30000DD07B68474A934207D07B68464A93426C
:100F400001D105230AE0062308E0042306E0032379
:100F500004E0022302E0012300E000237A69032178
:100F60000A40920093403A6913433B6135497B69DB
:100F70009B0802339B003A695A50384B9B683B618F
:100F8000FB68DA433B6913403B613B685A68802346
:100F90005B03134003D03A69FB6813433B612F4B5B
:100FA0003A699A602D4BDB683B61FB68DA433B6929
:100FB00013403B613B685A6880239B03134003D076
:100FC0003A69FB6813433B61244B3A69DA60234B6F
:100FD0005B683B61FB68DA433B6913403B613B68FC
:100FE0005A6880239B02134003D03A69FB6813437D
:100FF0003B611A4B3A695A60184B1B683B61FB68AE
:10100000DA433B6913403B613B685A6880235B02CB
:10101000134003D03A69FB6813433B610F4B3A69B5
:101020001A607B6901337B613B681A687B69DA402F
:10103000131E00D0A2E6C046C046BD4606B080BD25
:101040000010024000000140000400500008005061
:10105000000C005000100050001C00500004014023
:1010600080B584B000AF78600A00BB1C1A807B6832
:101070001B69BA1C1288134004D00F23FB180122ED
:101080001A7003E00F23FB1800221A700F23FB18BD
:101090001B781800BD4604B080BD0000B0B58AB012
:1010A00000AF78607B68002B02D1012300F0BFFB0A
:1010B000C94BDB680C221340FB61C74BDA68802305
:1010C0005B021340BB617B681B680122134000D1A7
:1010D0007EE0FB69082B07D0FB690C2B12D1BA69A3
:1010E00080235B029A420DD1BB4B1A6880239B027E
:1010F000134000D16BE07B685B68002B67D1012354
:1011000000F095FB7B685A6880235B029A4207D106
:10111000B14B1A68B04B802149020A431A6027E09C
:101120007B685A68A023DB029A420ED1AA4B1A6848
:10113000A94B8021C9020A431A60A74B1A68A64B23
:10114000802149020A431A6012E0A34B1A68A24B9D
:10115000A2490A401A60A04B1A6880235B02134020
:10116000FB60FB689C4B1A689B4B9D490A401A60C8
:101170007B685B68002B15D0FFF736FD03007B61B1
:1011800009E0FFF731FD02007B69D31A642B02D915
:10119000032300F04CFB904B1A6880239B02134002
:1011A000EFD015E0FFF720FD03007B6108E0FFF7BB
:1011B0001BFD02007B69D31A642B01D9032336E39C
:1011C000854B1A6880239B021340F0D100E0C04693
:1011D0007B681B680222134000D199E07B68DB68C2
:1011E0007B627B6A2022134009D07B4B1A687A4BC2
:1011F00020210A431A607B6A202293437B62FB69A9
:10120000042B05D0FB690C2B3ED1BB69002B3BD1D5
:10121000714B1B680422134004D07B6A002B01D160
:10122000012304E36C4B5B686E4A134019007B6832
:101230001B691A02684B0A435A60674B1B680922F4
:1012400093431900644B7A6A0A431A6000F042FC27
:101250000100614BDB681B090F221340624AD35C1B
:101260000A00DA40614B1A60614B1B6813257C1938
:101270001800FFF773FC030023707B191B78002B09
:1012800046D07B191B78D2E27B6A002B27D0524BC9
:101290001B680922934319004F4B7A6A0A431A606C
:1012A000FFF7A2FC03007B6108E0FFF79DFC020052
:1012B0007B69D31A022B01D90323B8E2464B1B6882
:1012C00004221340F1D0444B5B68464A1340190096
:1012D0007B681B691A02404B0A435A6018E03E4B78
:1012E0001A683D4B01218A431A60FFF77DFC030019
:1012F0007B6108E0FFF778FC02007B69D31A022BC0
:1013000001D9032393E2344B1B6804221340F1D12B
:101310007B681B681022134000D1A2E0FB69002B00
:1013200040D12D4B1A6880239B00134005D07B6869
:10133000DB69002B01D1012379E2274B5B682D4A41
:10134000134019007B685A6A234B0A435A60224BA8
:101350005B681B02190A7B681B6A1A061E4B0A434C
:101360005A607B685B6A5B0B0133802212029A40F1
:10137000194BDB681B090F210B401B49CB5CDA4082
:101380001A4B1A601A4B1B6813257C191800FFF7BB
:10139000E5FB030023707B191B78002B61D07B19C0
:1013A0001B7844E27B68DB69002B40D00A4B1A684B
:1013B000094B802149000A431A60FFF715FC03001E
:1013C0007B6119E0FFF710FC02007B69D31A022B46
:1013D00012D903232BE2C04600100240FFFFFEFF9C
:1013E000FFFFFBFFFFE0FFFFC03800080000002008
:1013F00004000020FF1FFFFFCA4B1A6880239B00D8
:101400001340DFD0C74B5B68C74A134019007B68A5
:101410005A6AC44B0A435A60C24B5B681B02190AE2
:101420007B681B6A1A06BF4B0A435A6019E0BD4B22
:101430001A68BC4BBD490A401A60FFF7D5FB030090
:101440007B6108E0FFF7D0FB02007B69D31A022B17
:1014500001D90323EBE1B34B1A6880239B001340AF
:10146000F0D17B681B680822134036D07B685B692B
:10147000002B19D0AB4B1A6DAA4B01210A431A65F8
:10148000FFF7B2FB03007B6108E0FFF7ADFB020052
:101490007B69D31A022B01D90323C8E1A14B1B6D31
:1014A00002221340F1D018E09E4B1A6D9D4B012192
:1014B0008A431A65FFF798FB03007B6108E0FFF79A
:1014C00093FB02007B69D31A022B01D90323AEE1FF
:1014D000944B1B6D02221340F1D17B681B680422E0
:1014E000134000D1AEE023203B1800221A708D4B30
:1014F0009A6B80235B05134009D18A4B9A6B894B09
:10150000802149050A439A633B1801221A70884BCF
:101510001A6880235B0013401AD1854B1A68844BEC
:10152000802149000A431A60FFF75EFB03007B61DC
:1015300008E0FFF759FB02007B69D31A642B01D93D
:10154000032374E17A4B1A6880235B001340F0D0C8
:101550007B689A6880235B009A4207D1714B1A6DB1
:10156000704B802149000A431A6531E07B689B6813
:10157000002B0CD16B4B1A6D6A4B6C490A401A65F3
:10158000684B1A6D674B6B490A401A6520E07B680F
:101590009A68A023DB009A420ED1624B1A6D614B10
:1015A0008021C9000A431A655E4B1A6D5D4B80218C
:1015B00049000A431A650BE05A4B1A6D594B5B49B7
:1015C0000A401A65574B1A6D564B5A490A401A651C
:1015D0007B689B68002B15D0FFF706FB03007B613F
:1015E00009E0FFF701FB02007B69D31A524A9342DC
:1015F00001D903231BE14B4B1A6D80239B00134041
:10160000EFD014E0FFF7F0FA03007B6109E0FFF789
:10161000EBFA02007B69D31A474A934201D90323AC
:1016200005E1404B1A6D80239B001340EFD123232B
:10163000FB181B78012B05D13A4B9A6B394B3F496C
:101640000A409A637B681B682022134049D07B685C
:101650009B69002B26D0334B9A68324B01210A43F9
:101660009A60304B5A6B2F4B01210A435A63344B1B
:101670001A6A334B802189010A431A62FFF7B4FAD0
:1016800003007B6108E0FFF7AFFA02007B69D31A21
:10169000022B01D90323CAE0224B9B68022213408C
:1016A000F1D01EE01F4B9A681E4B01218A439A60BD
:1016B000234B1A6A224B23490A401A62FFF794FA15
:1016C00003007B6108E0FFF78FFA02007B69D31A01
:1016D000022B01D90323AAE0124B9B68022213407C
:1016E000F1D17B689B6A002B00D19FE0FB690C2B3A
:1016F00000D178E07B689B6A022B59D1094B1A68AC
:10170000084B11490A401A60FFF76EFA03007B612B
:101710001CE0FFF769FA02007B69D31A022B15D986
:10172000032384E000100240FF1FFFFFFFFEFFFFC6
:1017300000700040FFFBFFFF88130000FFFFFFEF7A
:1017400000000140FFDFFFFFFFFFFFFE3A4B1A687A
:1017500080239B041340DCD1374BDB68374A1340AE
:1017600019007B68DA6A7B681B6B1A437B685B6BCA
:101770001A43314B0A43DA602F4B1A682E4B8021F3
:1017800049040A431A60FFF72FFA03007B6108E05F
:10179000FFF72AFA02007B69D31A022B01D903232F
:1017A00045E0254B1A6880239B041340F0D03DE0B0
:1017B000214B1A68204B22490A401A60FFF714FA9D
:1017C00003007B6108E0FFF70FFA02007B69D31A80
:1017D000022B01D903232AE0174B1A6880239B04AC
:1017E0001340F0D122E07B689B6A012B01D10123D9
:1017F0001DE0114BDB68BB61BA6980235B021A40B4
:101800007B68DB6A9A420FD1BA69F0239B031A40C6
:101810007B681B6B9A4207D1BA69C0231B041A402C
:101820007B685B6B9A4201D0012300E00023180023
:10183000BD460AB0B0BDC04600100240FFFF02FF27
:10184000FFFFFFFEB0B584B000AF786039607B6801
:10185000002B01D1012328E1964B1B680122134084
:101860003A689A421ED9934B1B6801229343190090
:10187000904B3A680A431A60FFF7B6F90300FB6021
:1018800009E0FFF7B1F90200FB68D31A8A4A9342D4
:1018900001D9032309E1874B1B68012213403A68F1
:1018A0009A42EED17B681B680222134009D0834B19
:1018B000DB68F022934319007B689A687F4B0A43E8
:1018C000DA607B681B680122134000D189E07B68E5
:1018D0005B68022B07D1794B1A6880239B02134067
:1018E00020D10123E1E07B685B68032B07D1734BB8
:1018F0001A6880239B04134014D10123D5E07B6830
:101900005B68012B06D16D4B1B680422134009D183
:101910000123CAE0694B1A6880239B00134001D160
:101920000123C2E0654BDB680322934319007B6807
:101930005A68624B0A43DA60FFF756F90300FB600E
:101940007B685B68022B11D109E0FFF74DF90200BB
:10195000FB68D31A584A934201D90323A5E0574B99
:10196000DB680C221340082BEFD13AE07B685B6800
:10197000032B11D109E0FFF737F90200FB68D31AF6
:101980004D4A934201D903238FE04C4BDB680C2274
:1019900013400C2BEFD124E07B685B68012B1BD13B
:1019A00009E0FFF721F90200FB68D31A424A93428B
:1019B00001D9032379E0414BDB680C221340042B4F
:1019C000EFD10EE0FFF710F90200FB68D31A3A4A94
:1019D000934201D9032368E0384BDB680C221340A3
:1019E000F0D1344B1B68012213403A689A421ED250
:1019F000304B1B680122934319002E4B3A680A436F
:101A00001A60FFF7F1F80300FB6009E0FFF7ECF85C
:101A10000200FB68D31A284A934201D9032344E009
:101A2000244B1B68012213403A689A42EED17B682E
:101A30001B680422134009D0204BDB68204A134066
:101A400019007B68DA681D4B0A43DA607B681B6803
:101A5000082213400AD0194BDB681A4A13401900B8
:101A60007B681B69DA00154B0A43DA6000F032F834
:101A70000100124BDB681B090F221340124AD35C92
:101A80000A00DA40114B1A60114B1B680B257C19B8
:101A90001800FFF763F8030023707B191B78002BF5
:101AA00002D07B191B7800E000231800BD4604B06B
:101AB000B0BDC04600200240881300000010024064
:101AC000FFF8FFFFFFC7FFFFC0380008000000203D
:101AD00004000020B0B58EB000AF4C4BDB68FB6259
:101AE000FA6A0C2313400C2B14D000D97BE0042B92
:101AF00002D0082B0BD076E0444B1B681022134019
:101B000002D0434B3B637CE0424B3B6379E0424B6A
:101B10003B6376E0FB6A9A0C0F231A403F4B9B5CB9
:101B2000BB62FB6A9A0D0323134001337B62374B80
:101B3000DA6880235B0213401AD0BB6ABB610023C2
:101B4000FB61354A0023B869F969FEF789FB020099
:101B50000B00100019007B6A3B6100237B613A692E
:101B60007B69FEF75DFB02000B0013007B6337E02F
:101B7000264B1B68102213401AD0BB6ABB6000239F
:101B8000FB60234A0023B868F968FEF769FB02008E
:101B90000B00100019007B6A3B6000237B603A68F1
:101BA0007B68FEF73DFB02000B0013007B6317E030
:101BB000BB6A180000231900164A0023FEF750FBE9
:101BC00002000B00100019007B6A1C0000231D009E
:101BD00022002B00FEF724FB02000B0013007B63A6
:101BE0007B6B3B630DE0094B5B685B0B072213408B
:101BF0003B623B6A0133802212029A4013003B632E
:101C0000C0463B6B1800BD460EB0B0BD0010024090
:101C100000093D000024F40000127A00D0380008CA
:101C200080B582B000AF78607B68002B01D10123C2
:101C300032E07B6839229B5CDBB2002B07D17B68EA
:101C40003822002199547B681800FEF7CFFE7B688C
:101C50003922022199547B681A687B680433190081
:101C6000100000F091FA7B683E22012199547B68B4
:101C70003A22012199547B683B22012199547B68C7
:101C80003C22012199547B683D22012199547B68B3
:101C900039220121995400231800BD4602B080BDAD
:101CA00080B582B000AF78607B68002B01D1012342
:101CB00032E07B6839229B5CDBB2002B07D17B686A
:101CC0003822002199547B68180000F029F87B68BD
:101CD0003922022199547B681A687B680433190001
:101CE000100000F051FA7B683E22012199547B6874
:101CF0003A22012199547B683B22012199547B6847
:101D00003C22012199547B683D22012199547B6832
:101D100039220121995400231800BD4602B080BD2C
:101D200080B582B000AF7860C046BD4602B080BDCD
:101D300080B584B000AF786039603B68002B08D173
:101D40007B683A229B5CDBB2013B5A1E9341DBB2BB
:101D50001FE03B68042B08D17B683B229B5CDBB215
:101D6000013B5A1E9341DBB213E03B68082B08D1BC
:101D70007B683C229B5CDBB2013B5A1E9341DBB289
:101D800007E07B683D229B5CDBB2013B5A1E93411E
:101D9000DBB2002B01D0012352E03B68002B04D1C1
:101DA0007B683A220221995413E03B68042B04D14A
:101DB0007B683B22022199540BE03B68082B04D13D
:101DC0007B683C220221995403E07B683D2202217A
:101DD00099547B681B6839680122180000F0D0FB19
:101DE0007B681A688023DB059A420ED07B681B68EB
:101DF000154A934209D07B681B68144A934204D069
:101E00007B681B68124A934211D17B681B689B68F0
:101E100007221340FB60FB68062B10D07B681B6811
:101E20001A687B681B6801210A431A6007E07B6817
:101E30001B681A687B681B6801210A431A6000232B
:101E40001800BD4604B080BD0004004000080140F9
:101E50000014014080B586B000AFF860B9607A60C8
:101E60001723FB1800221A70FB6838229B5C012B99
:101E700001D10223ADE0FB683822012199547B682F
:101E80000C2B00D176E07B680C2B00D995E07B68A9
:101E9000082B4ED07B68082B00D98EE07B68002B86
:101EA00003D07B68042B21D087E0FB681B68BA68ED
:101EB0001100180000F0C6F9FB681B689A69FB68FE
:101EC0001B6808210A439A61FB681B689A69FB68D2
:101ED0001B6804218A439A61FB681B689969BB6887
:101EE000DA68FB681B680A439A616BE0FB681B6851
:101EF000BA681100180000F0E1F9FB681B689A69E4
:101F0000FB681B68802109010A439A61FB681B6812
:101F10009A69FB681B6831490A409A61FB681B6833
:101F20009969BB68DB681A02FB681B680A439A61FF
:101F300048E0FB681B68BA681100180000F000FA5E
:101F4000FB681B68DA69FB681B6808210A43DA61D1
:101F5000FB681B68DA69FB681B6804218A43DA6145
:101F6000FB681B68D969BB68DA68FB681B680A43B1
:101F7000DA6127E0FB681B68BA681100180000F0FE
:101F80001FFAFB681B68DA69FB681B68802109017E
:101F90000A43DA61FB681B68DA69FB681B680F4952
:101FA0000A40DA61FB681B68D969BB68DB681A0202
:101FB000FB681B680A43DA6104E01723FB1801225F
:101FC0001A70C046FB683822002199541723FB1869
:101FD0001B781800BD4606B080BDC046FFFBFFFF62
:101FE00080B584B000AF786039600F23FB18002201
:101FF0001A707B6838229B5C012B01D10223BCE064
:102000007B683822012199547B6839220221995436
:102010007B681B689B68BB60BB6877229343BB608F
:10202000BB68584A1340BB607B681B68BA689A60FB
:102030003B681B6880229201934240D0802292012B
:10204000934200D988E080225201934200D188E077
:1020500080225201934200D97EE0702B18D000D923
:102060007AE0602B4FD000D976E0502B3BD000D9DE
:1020700072E0402B57D000D96EE0302B63D06BD884
:10208000202B60D068D8002B5DD0102B5BD063E094
:102090007B6818683B6899683B685A683B68DB68EE
:1020A00000F04EFA7B681B689B68BB60BB687722B8
:1020B0001343BB607B681B68BA689A6052E07B6818
:1020C00018683B6899683B685A683B68DB6800F0B1
:1020D00037FA7B681B689A687B681B688021C90196
:1020E0000A439A603EE07B6818683B6859683B6821
:1020F000DB681A0000F0AAF97B681B685021180001
:1021000000F004FA2EE07B6818683B6859683B6869
:10211000DB681A0000F0C8F97B681B6860211800B2
:1021200000F0F4F91EE07B6818683B6859683B686A
:10213000DB681A0000F08AF97B681B6840211800F0
:1021400000F0E4F90EE07B681A683B681B68190030
:10215000100000F0DBF905E00F23FB1801221A70D4
:1021600000E0C0467B683922012199547B683822FF
:10217000002199540F23FB181B781800BD4604B0AA
:1021800080BDC046FF00FFFF80B584B000AF78601F
:1021900039607B681B68FB607A688023DB059A42A4
:1021A0000BD07B68234A934207D07B68224A934234
:1021B00003D07B68214A934208D1FB687022934385
:1021C000FB603B685B68FA681343FB607A688023B6
:1021D000DB059A420BD07B68164A934207D07B6896
:1021E000154A934203D07B68144A934208D1FB6896
:1021F000134A1340FB603B68DB68FA681343FB60DB
:10220000FB68802293431A003B681B691343FB6001
:102210007B68FA681A603B689A687B68DA623B6898
:102220001A687B689A627B6801225A61C046BD4683
:1022300004B080BD000400400008014000140140CB
:10224000FFFCFFFF80B586B000AF786039607B6827
:102250001B6A012293431A007B681A627B681B6A1F
:102260007B617B685B683B617B689B69FB60FB68AB
:1022700070229343FB60FB6803229343FB603B683F
:102280001B68FA681343FB607B69022293437B61FE
:102290003B689B687A6913437B617B683A695A6043
:1022A0007B68FA689A613B685A687B685A637B6806
:1022B0007A691A62C046BD4606B080BD80B586B058
:1022C00000AF786039607B681B6A102293431A0064
:1022D0007B681A627B681B6A7B617B685B683B6119
:1022E0007B689B69FB60FB68134A1340FB60FB68DB
:1022F000124A1340FB603B681B681B02FA681343D9
:10230000FB607B69202293437B613B689B681B01D8
:102310007A6913437B617B683A695A607B68FA6823
:102320009A613B685A687B689A637B687A691A622B
:10233000C046BD4606B080BDFF8FFFFFFFFCFFFF1C
:1023400080B586B000AF786039607B681B6A1A4A36
:102350001A407B681A627B681B6A7B617B685B68DA
:102360003B617B68DB69FB60FB6870229343FB6029
:10237000FB6803229343FB603B681B68FA681343C6
:10238000FB607B690D4A13407B613B689B681B02C5
:102390007A6913437B617B683A695A607B68FA68A3
:1023A000DA613B685A687B68DA637B687A691A622B
:1023B000C046BD4606B080BDFFFEFFFFFFFDFFFF2C
:1023C00080B586B000AF786039607B681B6A1B4AB5
:1023D0001A407B681A627B681B6A7B617B685B685A
:1023E0003B617B68DB69FB60FB68154A1340FB605F
:1023F000FB68144A1340FB603B681B681B02FA68C9
:102400001343FB607B69104A13407B613B689B6808
:102410001B037A6913437B617B683A695A607B6866
:10242000FA68DA613B685A687B681A647B687A6983
:102430001A62C046BD4606B080BDC046FFEFFFFF32
:10244000FF8FFFFFFFFCFFFFFFDFFFFF80B586B0C0
:1024500000AFF860B9607A60FB681B6A7B61FB685B
:102460001B6A012293431A00FB681A62FB689B698E
:102470003B613B69F02293433B617B681B013A69F6
:1024800013433B617B690A2293437B617A69BB6892
:1024900013437B61FB683A699A61FB687A691A6247
:1024A000C046BD4606B080BD80B586B000AFF860BE
:1024B000B9607A60FB681B6A102293431A00FB68BC
:1024C0001A62FB689B697B61FB681B6A3B617B69E5
:1024D0000D4A13407B617B681B037A6913437B6160
:1024E0003B69A02293433B61BB681B013A691343DC
:1024F0003B61FB687A699A61FB683A691A62C04677
:10250000BD4606B080BDC046FF0FFFFF80B584B05A
:1025100000AF786039607B689B68FB60FB68702265
:102520009343FB603A68FB68134307221343FB6045
:102530007B68FA689A60C046BD4604B080BD000062
:1025400080B586B000AFF860B9607A603B60FB6828
:102550009B687B617B69094A13407B613B681A0277
:102560007B681A43BB6813437A6913437B61FB683A
:102570007A699A60C046BD4606B080BDFF00FFFF85
:1025800080B586B000AFF860B9607A60BB681F2282
:10259000134001229A4013007B61FB681B6A7A6931
:1025A000D2431A40FB681A62FB681A6ABB681F2193
:1025B0000B40796899400B001A43FB681A62C046C9
:1025C000BD4606B080BD000080B584B000AF786025
:1025D00039607B6838229B5C012B01D1022347E0E4
:1025E0007B683822012199547B6839220221995451
:1025F0007B681B685B68FB607B681B689B68BB60D3
:10260000FB6870229343FB603B681B68FA681343C6
:10261000FB607B681B68FA685A607B681A688023D5
:10262000DB059A420ED07B681B68134A934209D09F
:102630007B681B68114A934204D07B681B68104A70
:1026400093420CD1BB6880229343BB603B685B68BC
:10265000BA681343BB607B681B68BA689A607B6882
:102660003922012199547B68382200219954002392
:102670001800BD4604B080BD0004004000080140C1
:102680000014014080B584B000AF0200BB1D1A8069
:102690000023FB60BB1D00229B5E842B06D0BB1D6C
:1026A00000229A5EFB68D3180333FB60FB681800B6
:1026B000BD4604B080BD80B500AF00F0ADFA002388
:1026C0001800BD4680BDF0B589B004AF78603960B0
:1026D0007B685B69002B20D07B689B69002B1CD03A
:1026E0007B685C687B681D687B681E697B68082264
:1026F0009B5E1800FFF7C6FF7B685A697B689B6981
:1027000039680293019200900B00320029002000EA
:1027100000F0E3F80300FB601DE07B685C687B6809
:102720001D687B681B699EB27B6808229B5E18004F
:10273000FFF7A8FF01003A680C23FB1801930091F2
:10274000130032002900200000F00EF90300012BD5
:1027500001D0002300E0FB681800BD4605B0F0BDC5
:1027600080B584B000AF78607B68FB60FB68002BAD
:1027700001D0FB6800E00123180000F027FA0023D5
:102780001800BD4604B080BD80B582B000AF78604F
:102790007B6808331A007B685A607B6801225242CA
:1027A0009A607B6808331A007B68DA607B680833BC
:1027B0001A007B681A617B6800221A60C046BD4619
:1027C00002B080BD80B582B000AF78607B68002227
:1027D0001A61C046BD4602B080BD80B584B000AF6E
:1027E000786039607B685B68FB603B68FA685A60B8
:1027F000FB689A683B689A60FB689B683A685A6015
:10280000FB683A689A603B687A681A617B681B6863
:102810005A1C7B681A60C046BD4604B080BD80B5B6
:1028200084B000AF786039603B681B68BB60BB68F0
:10283000013303D17B681B69FB600CE07B680833C4
:10284000FB6002E0FB685B68FB60FB685B681B6821
:10285000BA689A42F6D2FB685A683B685A603B688D
:102860005B683A689A603B68FA689A60FB683A6805
:102870005A603B687A681A617B681B685A1C7B68DF
:102880001A60C046BD4604B080BD80B584B000AFBC
:1028900078607B681B69FB607B685B687A6892681C
:1028A0009A607B689B687A6852685A60FB685B68CC
:1028B0007A689A4203D17B689A68FB685A607B68A1
:1028C00000221A61FB681B685A1EFB681A60FB68CD
:1028D0001B681800BD4604B080BD90B58DB004AF34
:1028E000F860B9607A603B607B6B002B02D172B6F6
:1028F000C046FDE7BB6B002B02D172B6C046FDE7B8
:1029000054237B617B69542B02D072B6C046FDE72D
:102910007B69BB6B002B20D07B6B002B1DD0BB6B6E
:10292000FB61FB697A6B1A63FB695122022199549E
:102930003C687A68B968F86800230393FB690293DE
:102940001823FB1801933B6B0093230000F058F809
:10295000FB69180000F0D6F801E00023BB61BB69F9
:102960001800BD4609B090BD90B58DB004AFF860B9
:10297000B9603B60BB1D1A80BB1D1B889B00180003
:1029800000F09EFD03007B617B69002B10D054207A
:1029900000F096FD0300FB61FB69002B03D0FB698F
:1029A0007A691A6306E07B69180000F031FE01E0E5
:1029B0000023FB61FB69002B1AD0FB695122002127
:1029C0009954BB1D1A883C68B968F86800230393C2
:1029D000FB6902937B6B01933B6B0093230000F038
:1029E0000FF8FB69180000F08DF80123BB6102E0CD
:1029F00001235B42BB61BB691800BD4609B090BDB5
:102A000080B586B000AFF860B9607A603B60BB6AA1
:102A10001A6B7B683A498C4663449B00D3183B6130
:102A20003B69072293433B613B690722134002D075
:102A300072B6C046FDE7BB68002B20D000237B6147
:102A400013E0BA687B69D3181878BA6A34217B69B5
:102A5000D3185B18021C1A70BA687B69D3181B78EC
:102A6000002B06D07B6901337B617B690F2BE8D992
:102A700000E0C046BB6A43220021995403E0BB6AD0
:102A80003422002199543B6A062B01D906233B626C
:102A9000BB6A3A6ADA62BB6A3A6A5A64BB6A002263
:102AA0009A64BB6A04331800FFF78CFEBB6A1833C4
:102AB0001800FFF787FEBB6ABA6A1A613B6A0722F1
:102AC000D21ABB6A9A61BB6ABA6A5A62BB6A0022AE
:102AD000DA64BB6A5022002199543A68F9683B696C
:102AE000180000F0BBFB0200BB6A1A607B6A002B77
:102AF00002D07B6ABA6A1A60C046BD4606B080BD85
:102B0000FFFFFF3F80B582B000AF786000F040FC6F
:102B1000284B1B685A1C274B1A60274B1B68002B3D
:102B200009D1254B7A681A60224B1B68012B10D102
:102B300000F06AFA0DE0214B1B68002B09D11E4BF7
:102B40001B68DA6A7B68DB6A9A4202D81A4B7A6899
:102B50001A601B4B1B685A1C194B1A607B68DA6A97
:102B6000184B1B689A4203D97B68DA6A154B1A60C6
:102B70007B68DA6A13009B009B189B00124A9A1824
:102B80007B68043319001000FFF727FE00F012FCE9
:102B90000A4B1B68002B08D0074B1B68DA6A7B685E
:102BA000DB6A9A4201D200F0E3FBC046BD4602B0A8
:102BB00080BDC046D0030020D0020020DC030020EE
:102BC000EC030020D8030020D402002080B584B09C
:102BD00000AF78600023FB607B68002B11D00D4BA9
:102BE0001B68002B02D072B6C046FDE700F062F809
:102BF0007B680021180000F0DDFA00F067F80300A0
:102C0000FB60FB68002B01D100F0B2FBC046BD4663
:102C100004B080BDF803002090B589B004AF002354
:102C2000BB6000237B603A00391D0823FB181800A5
:102C3000FDF73AFC3C687B68BA681849184802926C
:102C400001930023009300232200FFF746FE0200B9
:102C5000144B1A60134B1B68002B02D00123FB603E
:102C600001E00023FB60FB68012B0DD172B60E4B17
:102C7000012252421A600D4B01221A600C4B0022B5
:102C80001A6000F051FB05E0FB68013302D172B617
:102C9000C046FDE7C046BD4605B090BDB838000847
:102CA000E92F0008F4030020F0030020DC030020DB
:102CB000D403002080B500AF034B1B685A1C024BA5
:102CC0001A60C046BD4680BDF803002080B584B0C0
:102CD00000AF0023FB600023BB603A4B1B68002B56
:102CE00002D172B6C046FDE700F052FB354B1B68BF
:102CF0005A1E344B1A60334B1B68002B5BD1324B8E
:102D00001B68002B57D02FE0304BDB68DB68FB6083
:102D1000FB6818331800FFF7B8FDFB680433180090
:102D2000FFF7B3FDFB68DA6A294B1B689A4203D9A7
:102D3000FB68DA6A264B1A60FB68DA6A13009B00AC
:102D40009B189B00234A9A18FB6804331900100053
:102D5000FFF743FDFB68DA6A1F4B1B68DB6A9A4288
:102D600002D31E4B01221A60184B1B68002BCBD1DB
:102D7000FB68002B01D000F0E3F9194B1B687B6066
:102D80007B68002B0FD000F02DF8031E02D0134BF0
:102D900001221A607B68013B7B607B68002BF2D1CB
:102DA0000F4B00221A600D4B1B68002B03D0012330
:102DB000BB6000F0DDFA00F0FDFABB681800BD460C
:102DC00004B080BDF8030020D00300209003002051
:102DD000D8030020D4020020D0020020E403002009
:102DE000E003002080B586B000AF00237B614A4B32
:102DF0001B68002B00D07FE0484B1B6801333B6110
:102E0000464B3A691A603B69002B18D1444B1B684A
:102E10001B68002B02D072B6C046FDE7404B1B6812
:102E2000FB60404B1A683E4B1A603E4BFA681A60D2
:102E30003D4B1B685A1C3C4B1A6000F081F93B4B20
:102E40001B683A699A4249D3354B1B681B68002BB3
:102E500004D1364B012252421A603FE0304B1B68CE
:102E6000DB68DB68BB60BB685B687B603A697B687A
:102E70009A4203D22D4B7A681A602FE0BB68043364
:102E80001800FFF702FDBB689B6A002B04D0BB68EB
:102E900018331800FFF7F9FCBB68DA6A244B1B688B
:102EA0009A4203D9BB68DA6A214B1A60BB68DA6AB6
:102EB00013009B009B189B001E4A9A18BB680433A2
:102EC00019001000FFF789FCBB68DA6A1A4B1B680F
:102ED000DB6A9A42B8D301237B61B5E7164B1B68C6
:102EE000DA6A144913009B009B189B005B58012B66
:102EF00007D901237B6104E0104B1B685A1C0F4B60
:102F00001A600F4B1B68002B01D001237B617B698A
:102F10001800BD4606B080BDF8030020D403002091
:102F2000880300208C030020E8030020F003002029
:102F3000D8030020D4020020D0020020E0030020AB
:102F4000E403002080B582B000AF224B1B68002B49
:102F500003D0214B01221A6038E01F4B00221A6077
:102F60001E4B1B687B6008E07B68002B02D172B6A9
:102F7000C046FDE77B68013B7B6019497A68130016
:102F80009B009B189B005B58002BEDD07A681300C8
:102F90009B009B189B00124A9B183B603B685B6838
:102FA0005A683B685A603B685A683B6808339A42E3
:102FB00004D13B685B685A683B685A603B685B6851
:102FC000DA68084B1A60054B7A681A60C046BD463D
:102FD00002B080BDF8030020E4030020D8030020E5
:102FE000D4020020D002002080B582B000AF78600B
:102FF00000F04EF8034B1B68012BF9D900F0B8F92B
:10300000F6E7C046D402002080B582B000AF0023AE
:103010007B600CE07A6813009B009B189B00144AAD
:103020009B181800FFF7B0FB7B6801337B607B685F
:10303000062BEFD90F4B1800FFF7A6FB0E4B18001D
:10304000FFF7A2FB0D4B1800FFF79EFB0C4B18007F
:10305000FFF79AFB0B4B1800FFF796FB0A4B054A4C
:103060001A600A4B044A1A60C046BD4602B080BDD1
:10307000D40200206003002074030020900300208D
:10308000A4030020BC030020880300208C03002040
:1030900080B582B000AF1AE000F07AF9104BDB681F
:1030A000DB687B607B6804331800FFF7EEFB0D4B99
:1030B0001B685A1E0B4B1A600B4B1B685A1E0A4B9F
:1030C0001A6000F077F97B68180000F00FF8064BE3
:1030D0001B68002BE0D1C046C046BD4602B080BD93
:1030E000A4030020D0030020B803002080B582B0E4
:1030F00000AF78607B6851229B5C002B09D17B6814
:103100001B6B180000F084FA7B68180000F080FA4E
:1031100011E07B6851229B5C012B04D17B68180075
:1031200000F076FA07E07B6851229B5C022B02D00C
:1031300072B6C046FDE7C046BD4602B080BD000085
:1031400080B582B000AF0B4B1B681B68002B04D10D
:10315000094B012252421A6008E0064B1B68DB68EB
:10316000DB687B607B685A68034B1A60C046BD46CB
:1031700002B080BD88030020F003002080B582B03B
:1031800000AF0A4B1B68002B02D101237B6008E0D3
:10319000074B1B68002B02D102237B6001E0002358
:1031A0007B607B681800BD4602B080BDDC03002058
:1031B000F803002080B584B000AF78603960214BFF
:1031C0001B68FB60204B1B6804331800FFF75DFB96
:1031D0007B6801330BD13B68002B08D01A4B1B686E
:1031E0001A1D1A4B11001800FFF7F7FA26E0FA68CB
:1031F0007B68D318BB60144B1B68BA685A60BA6806
:10320000FB689A4209D2124B1A680F4B1B680433B1
:1032100019001000FFF703FB10E00E4B1A680A4B71
:103220001B68043319001000FFF7F9FA0A4B1B68FA
:10323000BA689A4202D2084BBA681A60C046BD46C4
:1032400004B080BDD4030020D0020020BC030020C5
:103250008C03002088030020F003002080B584B098
:1032600000AFF860B9607A60FB68043BFB60FB6804
:10327000802252041A60FB68043BFB60BA68FB685A
:103280001A60FB68043BFB60084AFB681A60FB6835
:10329000143BFB607A68FB681A60FB68203BFB60AC
:1032A000FB681800BD4604B080BDC046B1320008BE
:1032B00080B582B000AF00237B60084B1B680133F0
:1032C00002D072B6C046FDE772B6C0467B68002BDE
:1032D000FCD0C046C046BD4602B080BD0C000020F8
:1032E00080B500AFC046BD4680BD000000000000B4
:1032F0000B4A13681868203080F30988022080F395
:103300001488BFF36F8F3FBCAE4608BC04BC62B6E6
:103310001847C046C046C046C046C046C046C04624
:10332000D0020020C046C04680B500AF0E4B1A68E0
:103330000D4BFF2109040A431A600B4B1A680A4B14
:10334000FF2109060A431A6000F098F8074B002293
:103350001A60FFF7CDFFFFF7F5FDFFF7A9FF002388
:103360001800BD4680BDC04620ED00E00C000020E6
:1033700080B500AF054B802252051A60BFF34F8F16
:10338000BFF36F8FC046BD4680BDC04604ED00E070
:1033900080B500AF72B6064B1B685A1C044B1A600E
:1033A000BFF34F8FBFF36F8FC046BD4680BDC04691
:1033B0000C00002080B500AF094B1B68002B02D128
:1033C00072B6C046FDE7064B1B685A1E044B1A60D6
:1033D000034B1B68002B00D162B6C046BD4680BDC2
:1033E0000C000020EFF3108072B67047C046180042
:1033F00080F310887047C046000000000000000005
:10340000EFF309800E4B1A6820381060F0C0444674
:103410004D4656465F46F0C008B572B6FFF792FDBE
:1034200062B60CBC116808681030F0C8A046A94606
:10343000B246BB4680F309882038F0C81847C0461A
:10344000D0020020C046C04680B582B000AFFFF772
:10345000C9FF03007B60FFF7C5FC031E03D0064BCA
:10346000802252051A607B681800FFF7C1FFC04632
:10347000BD4602B080BDC04604ED00E080B500AF9F
:103480000B4B00221A600B4B00221A600A4B1B6880
:10349000FA2291001800FCF737FE03001A00074BD0
:1034A000013A1A60024B07221A60C046BD4680BD31
:1034B00010E000E018E000E00000002014E000E070
:1034C00080B586B000AF78600023FB60FFF7F2FBA9
:1034D0004A4B1B68002B01D100F0E4F8484B1B68F5
:1034E0007A68134000D07BE07B68002B13D0082261
:1034F0007B689B187B607B68072213400BD07B683E
:103500000722934308337B607B680722134002D075
:1035100072B6C046FDE77B68002B61D0394B1B6853
:103520007A689A425CD8384B3B61374B1B687B61A9
:1035300004E07B693B617B691B687B617B695B683D
:103540007A689A4203D97B691B68002BF1D12B4B17
:103550001B687A699A4243D03B691B6808229B1812
:10356000FB607B691A683B691A607B695A687B68F3
:10357000D21A08235B009A4217D97A697B68D3185C
:10358000BB60BB680722134002D072B6C046FDE79D
:103590007B695A687B68D21ABB685A607B697A6813
:1035A0005A60BB68180000F0DDF8164B1A687B699A
:1035B0005B68D21A134B1A60124B1A68134B1B68C4
:1035C0009A4203D20F4B1A68104B1A607B695A68F3
:1035D0000B4B1B681A437B695A607B6900221A6097
:1035E000FFF774FBFB680722134002D072B6C04697
:1035F000FDE7FB681800BD4606B080BD0410002042
:103600001010002008100020FC0F00200C100020DB
:1036100080B584B000AF78607B68FB607B68002B6E
:1036200037D008235B42FA68D318FB60FB68BB60A5
:10363000BB685A68194B1B68134002D172B6C0466A
:10364000FDE7BB681B68002B02D072B6C046FDE7E1
:10365000BB685A68114B1B6813401AD0BB681B68C3
:10366000002B16D1BB685A680C4B1B68DB431A4011
:10367000BB685A60FFF71EFBBB685A68084B1B68A3
:10368000D218074B1A60BB68180000F06BF8FFF700
:103690001DFBC046BD4604B080BDC04610100020D2
:1036A0000810002080B584B000AFC0231B01BB60B0
:1036B000264BFB60FB68072213400CD0FB680733E6
:1036C000FB60FB6807229343FB60BA68FB68D21A71
:1036D0001E4BD318BB60FB687B601D4B7A681A6079
:1036E0001B4B00225A607B68BA68D318FB60082223
:1036F000FB689B1AFB60FB6807229343FB60FA6838
:10370000144B1A60134B1B6800225A60114B1B6844
:1037100000221A607B683B603B68FA68D21A3B68FB
:103720005A600C4B1A683B681A603B685A680A4B2F
:103730001A603B685A68094B1A60094B80221206CE
:103740001A60C046BD4604B080BDC046FC030020E0
:10375000FC0F0020041000200C1000200810002096
:103760001010002080B584B000AF7860274BFB605C
:1037700002E0FB681B68FB60FB681B687A689A4282
:10378000F7D8FB68BB60FB685B68BA68D3187A68D7
:103790009A4208D1FB685A687B685B68D218FB685C
:1037A0005A60FB687B607B68BB607B685B68BA685B
:1037B000D218FB681B689A4218D1FB681A68144B30
:1037C0001B689A420DD07B685A68FB681B685B686F
:1037D000D2187B685A60FB681B681A687B681A609D
:1037E00008E00B4B1A687B681A6003E0FB681A68F4
:1037F0007B681A60FA687B689A4202D0FB687A6834
:103800001A60C046BD4604B080BDC046FC0F002013
:103810000410002003008218934200D170471970F1
:103820000133F9E770B500260C4C0D4D641BA41054
:10383000A64209D1002600F019F80A4C0A4D641B73
:10384000A410A64205D170BDB300EB5898470136CD
:10385000EEE7B300EB5898470136F2E7E43800088A
:10386000E4380008E8380008E4380008F8B5C04635
:10387000F8BC08BC9E467047F8B5C046F8BC08BC0A
:043880009E467047A9
:10388400524742205461736B000000006465666116
:10389400756C745461736B009038000899090008C2
:1038A4000000000000000000800000000000000094
:1038B4000000000049444C450000000000000000E6
:1038C40000000000010203040607080903040608B7
:0838D4000C1018203000000068
:0838DC00E0C9FF7F01000000BC
:0438E400E9000008EF
:0438E800C100000813
:1038EC00000020000400000001000000AAAAAAAAFF
:0400000508000AC91C
:00000001FF
